:020000040000FA
:100000008B018A018301CA28F000030E8301F100ED
:100010000408F2008C1E4C28981C18194928181C3A
:1000200028283711B6011A08B100B7196328603AB9
:10003000031925283108320603194128A03A03196B
:100040002528603A03193C286328B5013715632831
:100050002030360784001A08371D63288000B50653
:10006000B60A20080F39023E3606031D63283711F1
:10007000B5080319B71563280614203099009900B4
:100080005A28371C6328061483160C168312B714DB
:1000900050281A08181218160C1E6328B71C5A2864
:1000A000A0303307840000089900B30AB40B63281A
:1000B0003710B7108316981C5B280C128312602827
:1000C00061286228061072088400710E8300F00E09
:1000D000700E090082073F3406345B344F346634B7
:1000E0006D347D3407347F346F343F0E0739820717
:1000F0000134023404340834103420344034803461
:1001000000348207013402340434083410342034BB
:100110004034003480348207013400340034003429
:1001200000348034403408341034820700341034F2
:100130002034403480340034003400340034BD199D
:10014000CF01CF08031908000301CF1A01304F1B5C
:100150000230CF180330CF0151078207122B5A2BE0
:10016000272B6D2B302B192B222B6D2B5E2B3C2B31
:10017000622B6D2B0800872B932BCA28872B722BA1
:100180007F2BCA28872BA12B9C2BCA28402B2C2BDA
:100190002A2B6D2B9801850186018316F630860087
:1001A000FF30850020308C00813081000B308E00C4
:1001B00000309F00831205309F00203084008001B2
:1001C000840A841FDF28851ABC17CF225D224724AA
:1001D000C623C0308B004030C900CA006E224D18C3
:1001E000452901305A24BF006030C10005220B218F
:1001F0003A210C183F213718F8280A220B215E23D8
:1002000000231C223C163A210C1C032911213A21FF
:10021000D1239F200729313090008E018F010C10CF
:10022000080090010C1008008C1C08008C109F1F07
:100230001E29C7304306031DC30A2129C308031D15
:10024000C303430C8400040C3F399500430E30393E
:100250000C3897004308C5070318C60AC40F0800E6
:100260004608C800C501C6013C170310CC0D031891
:100270004C14080014217922B7194B2108000C10E6
:10028000F930C9000730CA00080089233624142138
:1002900079229F2046292008613A031D7B292108E5
:1002A000031D5D29BD18032ABD11BD143D10F93091
:1002B000C9003F30CA00EE22012A013A031D6D2910
:1002C000BD11BD103D103F08D822EE223D080B396C
:1002D0000319012AB7111C22012A033A031D032A1C
:1002E000BD19032ABD15BD103D106D30C900733016
:1002F000CA00EE22012A033A031D8B292108223A63
:10030000031D032A2208BD00BD197529BD185729F0
:100310003D18A3296329013A031D97292108213A91
:10032000031D032A2208B8002308B900032A200865
:10033000813A031DA9292108031D032A3D18032A18
:10034000BD11BD103D14F930C9006D30CA00EE2258
:10035000012A2008E13A031DB8292108883A031D23
:10036000032A6D30C9004030CA00CC30CC00032ACB
:10037000033A031DC5292108F039203A031D032A39
:100380003C153F08BE00C101E529013A031DD829EB
:100390002108403A031D032A22083F39031D032A7E
:1003A00023083F06031D032A3C14EE223C16032AB1
:1003B000073A031DF5292108F039031D032A3C11D2
:1003C0003F08BE0023081F39C100A21BC116211C13
:1003D000A11841172119C11722087F39C0003C100C
:1003E000A1193C14EE223C16032A013A031D032AEC
:1003F0002108F039103A031D032A3C152508BE00D8
:10040000E229D101EE22B711080021304822213023
:100410005022592A2130482224305022592A803033
:100420004822592A2130482280305022592A21302E
:10043000482281305022592AE3304822003050228D
:10044000003050223F085022592AE4304822103010
:10045000411B1230C11B13305022003050223F0884
:1004600050224008C11A803850223C10EE223F082A
:10047000F30001306324592AE4304822203050220E
:10048000003050223F08502241081F395022352A9F
:10049000BA00B7194B213718492AB301B4013A08F9
:1004A000BB00A030340784003B088000B306B40AC8
:1004B0000800330850223714080000305A241F392E
:1004C000031901304038B2008400040E8406040C85
:1004D00084060419840A0418B2170800BC1B732A86
:1004E000851E0800752A851A08004B087720CD0460
:1004F00008000B1D08000B116E228316D9308504ED
:10050000F03086048312CA22CC1B0800F401F501E6
:100510004B0877204A0503198F2A0830B0224B0870
:10052000812049050319962A0730B022BC1BBE2240
:10053000BC1FC422CB08031D08004E094D05CF0087
:100540000319A42A3730D0004D08CE00CD014E0843
:1005500003190800D00B0800CF001630D0000800A7
:10056000F3008B20F40473089520F504080083162B
:10057000740985057509860583120800B722740879
:100580008504750886040800B72274098505750975
:1005900086050800CB0A09304B060319CB014B082E
:1005A0008B20F4004B089520F500BC1BC42ABE2A02
:1005B000CA0064304A020318EA2AC9010A30C90A8B
:1005C000CA020318DF2A4A076A20CA0049036A20C0
:1005D000C90008003830CA005C30E82A0301D1089D
:1005E000031D01303C18CC30BD18C3303D18C3305A
:1005F000BD19C330CC0008003F080F39043E080085
:10060000BC12FC225A24F30075207305031DBC168E
:100610000800FC225A24F3007520F304BC1EF306E4
:10062000602463343830C900CA010430D100EE229E
:10063000080009233F060319BF01BF0A00231C223B
:100640003F08D82A0923BF030319BF001E2B10300F
:10065000C1063C2A02302E2B01302E2BC1063C2233
:100660000830C1180130CA00083041180130C900F3
:100670001830D100EE2208002030C106BC06252229
:10068000C208031D5E2BC11E4E2B5E30C900083010
:10069000411B4030C11B0130CA00562B0830411BA2
:1006A0004030C11B0130C9005E30CA000830D100A3
:1006B000EE2208002030C106BC062522D101EE2220
:1006C0003F08D82AC208031D08008030C11F4030EF
:1006D000411BC030C1062522402B3D18172ABD18EA
:1006E0006E2B122A00305A24F300F30A20307306CE
:1006F00001300319F300003063247308D82A003056
:100700005A24F300F3031F300319F3007B2BBC1DA5
:100710008C2BBC1177308E2BBC157330C900CA01ED
:100720000C30D10008001430BC1D1030D100BC19B1
:10073000080000305A24D82A4808C700F3000230C5
:10074000632C831612088312F500F401083084002C
:10075000AE2B0310F40DF50D0318B22B48087502EB
:10076000031CB52B4808F5027414840BA92B7408DC
:10077000BC23F3000330632C8400841F041B31303E
:10078000841E3130831692008312080003305A24ED
:10079000BC233C3092000C30970002305A24C70032
:1007A00008003C1F08003C1337180800B71647081C
:1007B0000319E62B48020318DF2B003CB712FC3E5E
:1007C000031C030184000310840DE82B48088400F7
:1007D0003C1A252C411BFC2BC11B0C2C0310840C38
:1007E0000310840C0310840C0E3027240319080016
:1007F0002D24031D013E1B2C0310840C0310840CBC
:100800001C302724031908002D24031D033E8400F7
:10081000040C031810381B2C7E3027240319080001
:10082000C2060310420C2F24031D013ED108031DF4
:100830001B2C4218CA17C000C2080319252A3C08FD
:10084000370641062039C106252A3C120800040259
:10085000031884020408420608000408C200D108F4
:10086000031D342CD822CC01420808003C1F08008C
:100870003C135108143A031D08000310480CD822F9
:100880004818CA17480847060319C9170800061070
:10089000B701B601831603309900643098008312C3
:1008A000D03098000301FF3E031D532C1A081A088C
:1008B0001A08080083169B001C141A0883120800EB
:1008C00083165C24642C5A247306031908007308E9
:1008D00083169A001C158B1355309D00AA309D007D
:0E08E0009C148B171C119C18732C831208009B
:02400E00503F21
:104200000100030000003100000000000000000079
:10421000000000000000000000000000000000009E
:104220000000000000000000530069006D007000F5
:104230006C00650020004D006100750073002000D7
:1042400076002E0034000A0046002E004300610074
:10425000C300B1006100640061002D003E004A000F
:104260002E0046007500C4008D0069006B002D0013
:104270003E0048002E0048006100660074006D009A
:1042800061006E006E000A00310039002F0030001E
:0842900032002F003000350060
:00000001FF
